:02000000102FBF
:100E2000F9018301132F8B138312031385018601AC
:100E300087013B3083160313850070308600CE3067
:100E4000870004309100930170308F00803083124E
:100E500003179C0080309D001030831603139F0001
:100E6000831203130515E830F7000330F800780803
:100E70007704031D3C2F3D2F3E2F572F0330F100E9
:100E80009730F000F00B422FF10B422F472F8312C7
:100E90000313861786130130F7020030031CF80392
:100EA000F80278087704031D562F572F3E2F05119F
:100EB00087185B2F5C2FFE2F0630F1003030F000DA
:100EC000F00B602FF10B602F64008312031387185F
:100ED0006A2F6B2FF52F0515A730F4000030F500B1
:100EE00075087404031D752F762F772FE92F8F3027
:100EF0009F000330F1009730F000F00B7D2FF10BD5
:100F00007D2F822F832F831203139F18882F892F01
:100F1000832F1E080339F000F1010830FE00031092
:100F2000F00DF10DFE0B8F2F831603131E087007B3
:100F3000F2000030031801307107F3000030730233
:100F40000A30031972020318A62FA72FD42FD0300E
:100F5000F7000730F80078087704031DB02FB12F91
:100F6000B22FD42F83120313861700008613073085
:100F7000F0007008F600F608031DBF2FC02FC12F28
:100F8000C82F0130F602F608031DC72FC82FC12F46
:100F90000130F7020030031CF803F80278087704E8
:100FA000031DD32FD42FB22F0330F1009730F00060
:100FB000F00BD82FF10BD82FDD2F0130F4020030C9
:100FC000031CF503F50275087404031DE82FE92FCF
:100FD000772F8312031305110330F1009730F000CF
:100FE000F00BF02FF10BF02FF52F0330F1009730BD
:100FF000F000F00BF92FF10BF92FFE2F582F0028DE
:02400E00E4309C
:00000001FF
